:020000040800F2
:100000000000022035120008B5100008B7100008E3
:10001000B9100008BB100008BD1000080000000067
:10002000000000000000000000000000BF100008F9
:10003000C110000800000000C3100008C51000082F
:100040008512000885120008851200088512000834
:100050008512000885120008851200088512000824
:100060008512000885120008851200088512000814
:100070008512000885120008851200088512000804
:100080008512000885120008851200080000000093
:1000900000000000000000000000000085120008C1
:1000A0008512000885120008C91000088512000892
:1000B00085120008851200088512000885120008C4
:1000C00085120008851200088512000885120008B4
:1000D0008512000885120008851200080000000043
:1000E0008512000885120008851200080000000033
:1000F0000000000000000000000000008512000861
:100100000000000085120008851200088512000812
:1001100000000000000000000000000000000000DF
:100120008512000885120008851200088512000853
:100130008512000800000000000000000000000020
:100140000000000000000000000000008512000810
:100150008512000885120008851200088512000823
:100160008512000885120008000000000000000051
:10017000000000000000000000000000000000007F
:1001800000000000851200080000000000000000D0
:08019000851200088512000829
:1001980010B5054C237833B9044B13B10448AFF3B9
:1001A80000800123237010BD100000200000000013
:1001B800E012000808B5034B1BB103490348AFF32D
:1001C800008008BD0000000014000020E0120008B4
:1001D80053B94AB9002908BF00281CBF4FF0FF31A6
:1001E8004FF0FF3000F07AB9ADF1080C6DE904CE9C
:1001F80000F006F8DDF804E0DDE9022304B07047FA
:100208002DE9F0478C460D460446089E002B51D137
:100218008A4217466DD9B2FA82FEBEF1000F0BD0A2
:10022800CEF1200C01FA0EF520FA0CFC02FA0EF7BA
:100238004CEA050C00FA0EF44FEA174A250CBCFBF1
:10024800FAF81FFA87F90AFB18CC45EA0C4508FBAF
:1002580009F3AB420AD9ED1908F1FF3280F0238186
:10026800AB4240F22081A8F102083D44ED1AA4B245
:10027800B5FBFAF00AFB105544EA054400FB09F9FE
:10028800A14509D9E41900F1FF3380F00A81A1459D
:1002980040F2078102383C44A4EB090440EA0840D4
:1002A8000021002E61D024FA0EF40023346073601C
:1002B800BDE8F0878B4207D9002E54D0002186E88C
:1002C80021000846BDE8F087B3FA83F1002940F021
:1002D8008E80AB4202D3824200F2FA80841A65EB28
:1002E80003050120AC46002E3FD086E81010BDE87B
:1002F800F08712B90127B7FBF2F7B7FA87FEBEF10C
:10030800000F34D1EB1B3A0C1FFA87FC0121B3FB19
:10031800F2F8250C02FB183345EA03450CFB08F3F9
:10032800AB4207D9ED1908F1FF3002D2AB4200F217
:10033800D1808046ED1AA3B2B5FBF2F002FB10554E
:1003480043EA05440CFB00FCA44507D9E41900F175
:10035800FF3302D2A44500F2B8801846A4EB0C047F
:1003680040EA08409DE731463046BDE8F087CEF1C7
:10037800200405FA0EF307FA0EF720FA04F83A0CEF
:1003880025FA04F448EA0308B4FBF2F14FEA1845E9
:1003980002FB11441FFA87FC45EA044501FB0CF3F4
:1003A800AB4200FA0EF409D9ED1901F1FF3080F0E3
:1003B8008A80AB4240F2878002393D44EB1A1FFA2B
:1003C80088F5B3FBF2F002FB103345EA034500FB66
:1003D8000CF3AB4207D9ED1900F1FF386FD2AB42ED
:1003E8006DD902383D44EB1A40EA01418FE7C1F16B
:1003F800200722FA07F88B4005FA01F448EA0303BC
:1004080020FA07FE4FEA134CFD404EEA040EB5FBF6
:10041800FCF94FEA1E440CFB19551FFA83F844EA0D
:10042800054509FB08F4AC4202FA01F200FA01FAA8
:1004380008D9ED1809F1FF3043D2AC4241D9A9F1EE
:1004480002091D442D1B1FFA8EFEB5FBFCF00CFBA8
:1004580010554EEA054400FB08F8A04507D9E418F2
:1004680000F1FF3529D2A04527D902381C4440EABB
:100478000940A4EB0804A0FB02894C45C6464D463A
:1004880015D312D056B1BAEB0E0364EB050404FA87
:1004980007F7CB401F43CC40376074600021BDE8AC
:1004A800F0871846F8E69046E0E6C245EAD2B8EB8F
:1004B800020E69EB03050138E4E72846D7E7404612
:1004C80091E78146BEE7014678E702383C4445E7B4
:1004D800084608E7A8F102083D442BE7704700BF2B
:1004E80038B50E4A0E4B054618784FF47A73B3FBAD
:1004F800F0F31068B0FBF3F000F096F8044658B932
:100508000F2D09D8024629464FF0FF3000F04AF86F
:10051800044B20461D6038BD012038BD0C0000206A
:10052800000000200400002008B50B4B1A6842F4B4
:1005380000721A601A6842F480621A601A6842F4FB
:1005480080721A60032000F01BF80020FFF7C8FF34
:1005580000F072FD002008BD003C0240034A044B35
:1005680011681B780B441360704700BF30010020EE
:1005780000000020014B1868704700BF30010020C0
:10058800074AD36823F4E0631B041B0C43F0BF63E2
:10059800000243F4003300F4E0600343D360704783
:1005A80000ED00E0174B30B5DC68C4F30224C4F159
:1005B8000703251D042B28BF0423062D4FF0010532
:1005C80005FA03F303F1FF338CBF033C0024194001
:1005D800A14005FA04F4013C2240002842EA010245
:1005E8004FEA0212ADBF00F1604000F00F00064B69
:1005F80000F56140B5BFD2B2D2B21A5480F80023D8
:1006080030BD00BF00ED00E014ED00E0002808DB7D
:100618004209012300F01F0003FA00F0014B43F8E0
:100628002200704700E100E00138B0F1807F0AD273
:10063800064B074A5860F02182F823100020072251
:1006480098601A6070470120704700BF10E000E012
:1006580000ED00E02DE9F04F85B00B68DFF89C81D4
:10066800644A01934FF001090023019C09FA03F73A
:1006780007EA0406B74240F0AD804C6824F0100A3F
:10068800BAF1020F16D14FEAD30C00EB8C0C03F031
:10069800070BDCF820504FEA8B0B4FF00F0E0EFAC9
:1006A8000BFE25EA0E0E0D6905FA0BF545EA0E0557
:1006B800CCF820504FEA430C0325D0F800B005FAD7
:1006C8000CF5ED4304F0030E0BEA050B0EFA0CFED5
:1006D8000AF1FF3A4EEA0B0EBAF1010F0095C0F885
:1006E80000E015D8D0F808E005EA0E0ECD6805FA46
:1006F8000CFA4AEA0E0EC0F808E0D0F804E02EEA38
:100708000707C4F3001E0EFA03FE4EEA0707476008
:10071800C768009D3D408F6807FA0CF73D43C560E8
:10072800E50057D54FF0000BCDF80CB0D8F8447061
:10073800314D47F48047C8F84470D8F8447007F43E
:1007480080470397039F23F0030707F1804707F5C6
:100758009C3703F0030CD7F808A04FEA8C0C4FF035
:100768000F0E0EFA0CFEA8422AEA0E0E39D005F535
:100778008065A84237D005F58065A84235D005F5D3
:100788008065A84233D005F58065A84214BF0725C7
:10079800042505FA0CF545EA0E05BD601568F74312
:1007A80014F4803F0CBF3D4035431560556814F480
:1007B800003F0CBF3D4035435560956814F4801FD9
:1007C8000CBF3D4035439560D568A40254BF3D40F9
:1007D8003543D5600133102B7FF447AF05B0BDE832
:1007E800F08F5D46D5E70125D3E70225D1E703253C
:1007F800CFE700BF003C0140000002400038024043
:100808000AB1816170470904FBE7436931EA0303D0
:1008180008BF0904816170472DE9F341044618B9FE
:10082800012002B0BDE8F0810368DD0710D4236819
:10083800980758D423681A0700F19A8023685B0741
:1008480000F1B880A269002A40F019810020E8E789
:10085800A64B9A6802F00C02042A07D09A6802F0A4
:100868000C02082A0AD15B68590207D59F4B1B68FE
:100878009A03DCD56368002BD9D1D1E763689B4D17
:10088800B3F5803F11D12B6843F480332B60FFF719
:1008980071FE964D06462B689B03C8D4FFF76AFE87
:1008A800801B6428F7D90320BBE7B3F5A02F04D138
:1008B8002B6843F480232B60E5E72A6822F4803212
:1008C8002A602A6822F480222A60002BDFD1FFF7F1
:1008D80051FE06462B689F03A9D5FFF74BFE801BE8
:1008E8006428F7D9DFE7814B9A6812F00C0F07D01C
:1008F8009A6802F00C02082A11D15B685E020ED4D5
:100908007A4B1A68950702D5E268012A88D11A68D5
:10091800216922F0F80242EAC1021A608AE7E26815
:10092800734BB2B101221A60FFF724FE6F4D0646E1
:100938002B68980707D52B68226923F0F80343EA48
:10094800C2032B6076E7FFF715FE801B0228EFD95C
:10095800A9E71A60FFF70EFE644D06462B68990753
:100968007FF568AFFFF706FE801B0228F6D99AE7E5
:100978006269604B7AB101221A60FFF7FBFD5B4D9B
:1009880006466B6F9F073FF559AFFFF7F3FD801BD6
:100998000228F6D987E71A60FFF7ECFD534D0646A3
:1009A8006B6F98077FF54AAFFFF7E4FD801B0228BD
:1009B800F6D978E74D4B1A6C12F0805228D1019283
:1009C8001A6C42F080521A641B6C03F08053019336
:1009D800019B0126484D2B68D9051BD5A368434DBB
:1009E800012B27D12B6F43F001032B67FFF7C2FDC3
:1009F8003E4D074641F288382B6F9B0739D5002EAC
:100A08003FF420AF394A136C23F08053136419E77D
:100A18000026DFE72B6843F480732B60FFF7AAFDFD
:100A280007462B68DA05D9D4FFF7A4FDC01B0228B6
:100A3800F7D938E7052B04D12B6F43F004032B6754
:100A4800D0E72A6F22F001022A672A6F22F00402F7
:100A58002A67002BCAD1FFF78DFD41F28838074677
:100A68002B6F9807CBD5FFF785FDC01B4045F7D9FD
:100A780019E7FFF77FFDC01B4045BDD913E71B4DA4
:100A8800AB6803F00C03082B3FF4CAAE1B4E0023DF
:100A9800022A336034D1FFF76DFD07462B689901B0
:100AA8001ED4226AE3691343626A43EA8213E26A44
:100AB80043EA0263A26A0D4C5208013A43EA024330
:100AC8006B6001233360FFF755FD054623689A01E3
:100AD8003FF5BCAEFFF74EFD401B0228F6D9E2E613
:100AE800FFF748FDC01B0228D8D9DCE600380240D1
:100AF80000004742800E47420070004060004742B5
:100B0800FFF738FD04462B689B017FF59FAEFFF782
:100B180031FD001B0228F6D9C5E600BF134908B508
:100B28008B6803F00C03042B03D0082B03D0104868
:100B380008BD104808BD4A684B68496813F480032B
:100B480014BF0C480A48C1F3881118BF002302F0EB
:100B58003F02A1FB0001FFF73BFB044B5B68C3F3BB
:100B6800014301335B00B0FBF3F008BD00380240DD
:100B78000024F40000127A002DE9F0410D460446E5
:100B880010B90120BDE8F081444B1A6802F00F0249
:100B98008A4228D321688F072DD4C80740D43F4BF9
:100BA8001A6802F00F02954266D3226851076CD486
:100BB800130707D53A4A2169936823F4604343EA47
:100BC800C1039360FFF7AAFF354B364A9B68C3F30E
:100BD8000313D35CD840344B18600020FFF780FC27
:100BE8000020BDE8F081CAB21A701B6803F00F0339
:100BF8009942C6D1CEE72A4B11F0040F1EBF9A685E
:100C080042F4E0529A600E0742BF9A6842F460428A
:100C18009A609A68A06822F0F00202439A60BCE7E2
:100C280062681F4B012A1DD11B6813F4003FA8D02E
:100C38001B4EB36823F003031343B360FFF79AFC1A
:100C480041F288380746B368626803F00C03B3EBD7
:100C5800820FA4D0FFF78EFCC01B4045F3D90320B8
:100C6800BDE8F081911E01291B6802D813F0007FAE
:100C7800DDE713F0020FDAE7EAB21A701B6803F037
:100C88000F039D427FF47DAF8FE70549E0688B68CD
:100C980023F4E05303438B608AE700BF003C024023
:100CA80000380240F81200080C0000200368DA68D7
:100CB80042F00102DA609A6802F00702062A1EBFB3
:100CC8001A6842F001021A600020704770477047A6
:100CD8007047704703681A69910710B504460ED526
:100CE800DA6892070BD56FF002021A619B6901223C
:100CF8009B07027777D0FFF7EAFF00232377236863
:100D08001A69500710D5DA6851070DD56FF004023B
:100D18001A619B69022213F4407F2277204668D02B
:100D2800FFF7D5FF0023237723681A6912070FD529
:100D3800DA6810070CD56FF008021A61DB69042223
:100D48009907227720465AD0FFF7C1FF002323775F
:100D580023681A69D20610D5DA68D0060DD56FF067
:100D680010021A61DB69082213F4407F22772046BB
:100D78004BD0FFF7ACFF0023237723681A69D1070C
:100D880008D5DA68D20705D56FF001021A61204646
:100D980000F050F923681A69100608D5DA681106B8
:100DA80005D56FF080021A61204600F09EF823688E
:100DB8001A69520608D5DA68500605D56FF0400260
:100DC8001A612046FFF785FF23681A69910622D524
:100DD800DA6892061FD56FF0200220461A61BDE836
:100DE800104000F081B8FFF771FF2046FFF770FF51
:100DF80083E7FFF76BFF2046FFF76AFF92E7FFF7ED
:100E080065FF2046FFF764FFA0E7FFF75FFF204676
:100E1800FFF75EFFAFE710BD244A036890420ED08B
:100E2800B0F1804F0BD0A2F57C42904207D002F57A
:100E38008062904203D002F58062904215D14A68E0
:100E480023F070031343194A904219D0B0F1804F30
:100E580016D0A2F57C42904212D002F580629042F0
:100E68000ED002F5806290420AD0114A904207D013
:100E780002F58062904203D002F58062904203D16D
:100E8800CA6823F4407313434A6923F08003134369
:100E980003608B68C3620B688362044B984204BF8B
:100EA8000B69036301234361704700BF00000140E1
:100EB8000040014010B50446A0B190F83D3003F061
:100EC800FF021BB980F83C2000F0D2F8022384F816
:100ED8003D302068211DFFF79FFF012384F83D3036
:100EE800002010BD012010BD704770474FF400511D
:100EF8000148FFF78ABC00BF000C024070B594B0EF
:100F08003022002108A800F0DFF90021142203A8EC
:100F180000F0DAF900241A4B01941A6C42F080525E
:100F28001A641B6C03F080530193019B154B0294C8
:100F38001A6842F440421A601B680F9403F4404355
:100F48000293029B10230225C02201260C9308A8B5
:100F58000823109311921293139308950B960E95EC
:100F6800FFF75AFC0F23039331464FF4A05303A80D
:100F78000495059406930793FFF7FEFD14B070BD22
:100F8800003802400070004000B589B0FFF7CCFA85
:100F9800FFF7B4FF1422002103A800F095F90024FC
:100FA8001E4B02941A6B1E481E4D42F008021A632B
:100FB8001B6B03F00803224602934FF40051029B77
:100FC8000126FFF71DFC03A94FF4005314480393AF
:100FD800049605940694FFF73DFB134AAC6042F66D
:100FE800E063284685E80C00EE602C61AC61FFF7F1
:100FF80061FF284600F090F82846FFF757FE00F0FA
:10100800A1F80A4D0A4A2870234600944FF47A71D1
:1010180000F0A8F8287800F0BDF8FEE70038024094
:10102800000C024034010020004801400800002064
:10103800F50E000800F0D4B882B00C4B00210091E6
:101048005A6C42F480425A645A6C02F4804200920C
:10105800009A01911A6C42F080521A641B6C03F0DA
:1010680080530193019B02B0704700BF00380240D3
:1010780007B50D4B02689A4213D1002203F570435D
:101088000192596C41F4802159645B6C03F480230C
:1010980001931A201146019BFFF784FA1A20FFF7E3
:1010A800B5FA03B05DF804FB004801407047FEE75D
:1010B800FEE7FEE7FEE7704770477047FFF74EBA56
:1010C8000148FFF707BE00BF340100200F49D1F8DF
:1010D800883043F47003C1F888300D4B1A6800203B
:1010E80042F001021A6098601A6822F0847222F4B1
:1010F80080321A60074A5A601A6822F480221A60FD
:10110800D8604FF000638B60704700BF00ED00E0CF
:101118000038024010300024084B1860084B0022A9
:1011280003F580711A705A709A70DA709A80DA80B2
:101138009A601A7310338B42F4D170472C00002048
:1011480030000020064B00200201D15C19B90121B2
:101158009954C0B2704701301028F5D1F9E700BFA3
:1011680030000020102870B505460FD8084E000141
:101178003418305C58B100262373E5709DF81030A0
:101188006670A680E180A260A37070BD002070BD6B
:1011980030000020084A0301D118D35C2BB14A78EB
:1011A8002AB90F2805D801224A701846704700232B
:1011B800FBE71346F9E700BF30000020074A0301A8
:1011C800D118D35C3BB14B782BB10F284FF00002FC
:1011D80094BF4A7013461846704700BF300000207D
:1011E80038B5104B02681B681B689A4216D10E4C22
:1011F800002523786BB163785BB1A388E2889A42B3
:101208000DD8A368E0789847A3784BB1E8B2FFF708
:10121800D5FF0135102D04F11004EAD138BD013392
:10122800A380F6E72C00002030000020DFF834D03F
:10123800002103E00C4B5B58435004310B480C4B26
:1012480042189A42F6D30B4A02E0002342F8043BC4
:10125800094B9A42F9D3FFF739FF00F011F8FFF76D
:1012680093FE7047000002201813000800000020B9
:10127800100000201000002074010020FEE700008C
:1012880070B50D4E0D4CA41BA4100025A54209D124
:101298000B4E0C4C00F020F8A41BA4100025A5420E
:1012A80005D170BD56F8253098470135EEE756F858
:1012B800253098470135F2E710130008101300088D
:1012C800101300081413000802440346934200D187
:1012D800704703F8011BF9E7F8B500BFF8BC08BC74
:1012E8009E467047F8B500BFF8BC08BC9E467047DC
:1012F80000000000000000000102030406070809BE
:0813080000EFFF7F010000006F
:04131000BD01000813
:041314009901000833
:101318000100000010000000FF0000000024F4009D
:0400000508001235A8
:00000001FF
